:040000006F00F00895
:100004000000000000000000EE050000F005000004
:10001400000000008C080000000000000000000048
:100024008C0800008C0800000000000000000000A4
:100034007015000000000000000200000000000035
:100044008C0800008C0800008C0800008C0800005C
:100054008C0800008C0800008C0800008C0800004C
:100064008C0800008C0800008C0800008C0800003C
:100074008C0800008C0800008C0800008C0800002C
:100084008C0800008C0800008C0800008C0800001C
:100094008C0800008C0800008C0800008C0800000C
:1000A4008C0800008C0800008C0800008C080000FC
:1000B4008C0800008C0800008C0800008C080000EC
:1000C4008C0800008C0800008C0800008C080000DC
:1000D4008C0800008C080000083100005231000038
:1000E4008C0800008C0800008C0800008C080000BC
:1000F4008C0800008C0800008C0800008C080000AC
:10010400000000008C0800008C0800008C0800002F
:100114008C0800009C3100008C0800008C08000052
:100124008C0800008C0800008C0800008C0800007B
:100134008C0800008C0800008C0800008C0800006B
:100144008C0800008C0800008C0800008C0800005B
:100154008C0800008C0800008C080000E6310000C8
:10016400303200007A3200008C0800008C08000055
:100174008C0800008C0800008C0800008C0800002B
:100184008C0800008C0800008C0800008C0800001B
:100194008C0800008C0800008C0800008C0800000B
:1001A400000000000000000000000000000000004B
:0C01B4000000000000000000000000003F
:10020000130181F806C216C41AC61EC822CA26CC1B
:100210002ACE2ED032D236D43AD63ED842DA46DC76
:100220004ADECEC0D2C2D6C4DAC6DEC8E2CAE6CC46
:10023000EACEEED0F2D2F6D4FAD6FED8F3220030CF
:1002400096DA9702002083A222F723A02200F3254A
:1002500010342EC09305000273A0458003A1818154
:10026000EF10707117030020032303F5032103002F
:10027000824273901234D652739002309240A2425E
:100280003243C2435244E244724582551256A2564A
:100290003257C2575258E25872598649164AA64AEE
:1002A000364BC64B564CE64C764D865D165EA65ECA
:1002B000365FC65F13018107730020301300000012
:1002C00013000000130000001300000013000000E2
:1002D00013000000130000001300000013000000D2
:1002E00013000000130000001300000013000000C2
:1002F00013000000130000001300000013000000B2
:1003000083A28181938202E073900234170100205E
:10031000032181EA024182403243C2435244E24413
:10032000724582551256A2563257C2575258E25859
:1003300072598649164AA64A364BC64B564CE64C6D
:10034000764D865D165EA65E365FC65FD652A1020A
:1003500073900230A24213018107828013000000D3
:100360001300000013000000130000001300000041
:100370001300000013000000130000001300000031
:100380001300000013000000130000001300000021
:100390001300000013000000130000001300000011
:1003A0001300000013000000130000001300000001
:1003B00013000000130000001300000013000000F1
:1003C00013000000130000001300000013000000E1
:1003D00013000000130000001300000013000000D1
:1003E00013000000130000001300000013000000C1
:1003F00013000000130000001300000013000000B1
:10040000F322003093F272FF130380781203B3E2F9
:100410006200711523205500130585FA10C12115BE
:10042000232005009302000063870200711523203A
:100430000500FD12D5BF71150CC1828000000000BF
:1004400000000000000000000000000000000000AC
:10045000000000000000000000000000000000009C
:10046000000000000000000000000000000000008C
:10047000000000000000000000000000000000007C
:10048000000000000000000000000000000000006C
:10049000000000000000000000000000000000005C
:1004A000000000000000000000000000000000004C
:1004B000000000000000000000000000000000003C
:1004C000000000000000000000000000000000002C
:1004D000000000000000000000000000000000001C
:1004E000000000000000397101436EC619A0397187
:1004F00041536AC866CA62CC5ECE19A039710153F5
:100500005AD056D252D44ED64AD826DA22DC06DE4B
:1005100033016140828241114AC026C222C406C60C
:100520008282B24D4101024D924C224CB24B4101AC
:10053000024B924A224AB249410102499244224462
:10054000B240410182803D432A876373C30293779F
:10055000F700BDEFADE5937606FF3D8ABA960CC372
:100560004CC30CC74CC74107E36BD7FE11E2828036
:10057000B306C3408A069702000096966780A600DD
:100580002307B700A306B7002306B700A305B700EB
:100590002305B700A304B7002304B700A303B700E3
:1005A0002303B700A302B7002302B700A301B700DB
:1005B0002301B700A300B7002300B700828093F5A2
:1005C000F50F93968500D58D93960501D58D61B76E
:1005D000939627009702000096968682E78086FA17
:1005E0009680C1171D8F3E96E374C3F8A5B701A08E
:1005F000B707EFBE37E700E0938707083CC701A0C5
:10060000EFF27FF10945EF007009912AEF20401EBB
:10061000716513050520EF20C020B707002083A5D2
:1006200007173755000013058528EF30F022CD233A
:10063000AA853755000013058529EF30F021B755FD
:100640000000375500009385852A1305052BEF30F0
:10065000B020EF30C04E375400001305042DEF30AA
:10066000F030E5BFB71702409843B706FFF04111DD
:100670001367170098C3D84337060200758FD8C395
:100680009843B706F7FEFD16758F98C39843B706D3
:10069000FCFFFD16758F98C3D843B70601FFFD1602
:1006A000758FD8C39843B70600ECFD16758F98C3B5
:1006B0003707FF0098C723A6070202C402C6984363
:1006C000C166558F98C3B716024005679C42F18FEB
:1006D0003EC6A24785073EC4B24781E7A247E397DB
:1006E000E7FEB71702409C431397E70063570706DE
:1006F00085473EC632478547631FF704B717024058
:10070000D843B706C1FFFD16D8C3D843D8C3D843D2
:1007100013670740D8C3D843758FD8C3D843B706EB
:100720001100558FD8C39843B7060001558F98C361
:10073000984393166700E3DD06FED843B7160240E0
:10074000719BD8C3D84313672700D8C32147DC4225
:10075000B18BE39EE7FE4101828002C661BFB716FE
:100760000240D842B70700201146318B9387071704
:100770006305C70021466308C70237177A001307CD
:10078000072098C337170240584311839376F70028
:100790003707002013070700369714239843335771
:1007A000D70098C38280D842D442416649833D8BAA
:1007B000F18E1306270015CF3D47630FE602414730
:1007C000630FE602454781456313E6004146A1E217
:1007D0003747024003270780418B0DC737177A0040
:1007E000130707203306C70290C3C9DD984305836A
:1007F00049BF81454946E1BF85453546C9BF814569
:100800003D46F1B737173D0013070790E1BF371595
:10081000024058559316F700585563DF06041183BC
:100820003D8B9306170037177A00130707203357BD
:10083000D70298C35455A182BD8A8DE295463307ED
:10084000D702058398C337170240585794433D8B0E
:10085000050733D7E60298C3984369B70545639403
:10086000A600E546E9BF3D456396A600D14633871D
:10087000E602C9BF8906E5BF3D8B9306170037170F
:100880007A00130707203357D702F1B701A0970169
:1008900000209381210E177100201301A1761755B6
:1008A0000000130525D897F5FF1F9385A5751386BE
:1008B000018263FAC5008322050023A055001105BB
:1008C0009105E3EAC5FE170500201305A58C9735B1
:1008D00000209385E5F86377B50023200500110516
:1008E000E36DB5FEFD42739002BCFD427390428001
:1008F000B7820000938202807390023097F2FFFF6C
:100900009382827093E2320073905230EFF09FD561
:1009100097020000938202CF73901234730020304C
:10092000EFF27FBFB727014093870740631BF500B5
:100930008545130500205527814513050020712F9B
:10094000EDBEB737014093870780E31BF5FE854571
:10095000130500405927814513050040CDB75C4180
:100960003707F1E01307F7EF944D7D8F9C41D58F4A
:10097000D44DD58FD441A206D58FD98F5CC11C45EB
:1009800037F7F1FF1307D77FD4457D8F9C49D58F6B
:1009900094458606D58FD98F1CC55C55370710FF47
:1009A0007D177D8FDC29FD1793F7F70FD207D98FBD
:1009B0005CD582801C4589C593E717001CC58280E1
:1009C000F99BEDBF1C4589C593E707101CC58280C4
:1009D00093F7F7EFE5BF1C4593E787001CC58280BE
:1009E00008450D81058982801C4593E747001CC599
:1009F000828008450981058982801C4591C5370799
:100A00005000D98F1CC582803707B0FF7D17F98F42
:100A1000D5BFA54763F7B7048D47138765FF330735
:100A2000F7020328C5009D47B397E70093C7F7FF78
:100A3000B3F70701B396E600DD8E54C5994763E32B
:100A4000C70495477D163306F6025859FD47B397FC
:100A5000C70093C7F7FFF98F3396C5005D8E50D955
:100A600082800D473387E502032805019D47B39730
:100A7000E70093C7F7FFB3F70701B396E600DD8EF3
:100A800014C96DBFB14763E2C702954765163306C7
:100A9000F6021859FD47B397C70093C7F7FFF98FC0
:100AA0003396C5005D8E10D9828095474D1633066A
:100AB000F6025855FD47B397C70093C7F7FFF98F64
:100AC000B395C500DD8D4CD582805C4191C537075B
:100AD0000004D98F5CC18280370700FC7D17F98F35
:100AE000D5BFEFF25FA301112A8423040100A544BE
:100AF0001C8463F8F40423040100A54621461C84E9
:100B000063FCF606231501002304010095461C84AE
:100B100063FEF60C38853C8599460D46B3F7D7023F
:100B2000056513050580B3D7C7023357D702BA97B7
:100B3000C207C1837C853C8505611D8D42054185C9
:100B4000EDBA1C4493E787001CC42285513D75FD16
:100B50001C4493E747001CC42285613D75FD784421
:100B60001C8414108607B6972396E7FE1C8485071D
:100B700093F7F70F5C84ADBFA30401009C846378F6
:100B8000F6001C84850793F7F70F5C848DBF98846B
:100B90009C840C100607850786072E97AE9703578F
:100BA000C7FE83D7C7FE63FDE7029C848607AE9726
:100BB00083D7C7FE7C859C84988485078607AE977B
:100BC00083D5C7FE931717001810BA972396B7FE60
:100BD0009C8438850C1085078607AE972396E7FE20
:100BE0009C84850793F7F70FDC8449BF1C841010A1
:100BF000388589078607B29783D7C7FEBA97C20799
:100C0000C1837C851C84850793F7F70F5C8401B74B
:100C1000B7F7FF1F03A5477082801C414167791712
:100C2000F98F1CC123200500232205002324050081
:100C3000B707024023260500138787006317E500E6
:100C4000D8431367F700D8C382801387C7016316A0
:100C5000E500D8431367070FFDB713870703631831
:100C6000E500D8438566938606F0558FE9BF138764
:100C700047046315E500D843BD66C5BF13878705E4
:100C80006316E500D843B7060F00C5B71387C7063C
:100C90006316E500D843B706F000C1BF1387070805
:100CA0006316E500D843B706000FC1B71387874026
:100CB0006319E50003A747401367F70023A2E74045
:100CC00082801387C7416317E50003A74740136776
:100CD000070FEDB793870743631BF500B707024083
:100CE00003A747408566938606F0558FC1BFB707B7
:100CF0000240138747446316E50003A74740BD66DB
:100D0000EDB7138787456317E50003A74740B7068C
:100D10000F00E1BF1387C7466317E50003A74740ED
:100D2000B706F000D9B7138707486317E50003A794
:100D30004740B706000F55BF138707496319E50001
:100D400003A7474D1367F70023AAE74C8280138758
:100D5000074A6317E50003A7474D1367070FEDB771
:100D60001387074B6319E50003A7474D85669386F4
:100D700006F0558FD1BF1387074CE319E5FC03A795
:100D8000474DBD66FDB71C4161773D0794517D8F8E
:100D90009C45D58F9449D58FD449D58F944DD58F07
:100DA000D44DD58FD451D58F9455D58FD98F1CC1A3
:100DB000DC455CC19C411CC5DC415CC582801C419A
:100DC00089C593E717001CC1828041677917F98FA5
:100DD000DDBF9C4513F7070113F8F70001C7D841A1
:100DE0003368E8008E2113F7F50F39C318418146A7
:100DF000854E3D4F930F800293028004214E33961F
:100E0000DE00B3F8C5006311160393982600331370
:100E10001F011343F3FF3377E300B318180133E7DF
:100E2000E800639FF70550C98506E39AC6FD18C11F
:100E30001307F00F6375B70454412146854E3D4FAB
:100E4000930F800293028004414EB398CE0033F793
:100E500015016392E8021317260001173313EF0000
:100E60001343F3FFB376D3003317E800D98E639DA5
:100E7000F701232A15010506E319C6FD54C1828036
:100E8000E39457FA10C94DB7E39757FE232815018D
:100E9000DDB719C20CC982804CC98280B707002017
:100EA00023A8A7188280B707002003A7071989473E
:100EB00010216311F70214318D4763EDD7003C21F7
:100EC0009A0637E700E09607D58F93F7F70F32972A
:100ED0002300F74054410547935756003317C70086
:100EE00089CA938707048A07B7E600E0B69798C3D4
:100EF000828093870706C5BFB7160240DC42517750
:100F00007D17F98F5D8DC8C28280371702405C4320
:100F10009146B18B6385D700A1466382D706B71788
:100F20007A00938707201CC1371602405C423707BE
:100F30000020130707019183BD8BBA9794231C41AE
:100F4000B3D7D7005CC15442A1829D8ABA9694223D
:100F5000B3D6D70014C55442AD829D8A3697182364
:100F6000B3D7E7005CC558423983937637001387BF
:100F7000418036971823B3D7E7021CC982805C43AF
:100F80005843C166C983758FB7F6FF1F83A6C67025
:100F9000BD8B89071396160163480600C5460146B6
:100FA0006392D702C94739A88946638FD702BD46E5
:100FB000638ED702C146638ED702C546014663934E
:100FC000D700C1471DEF3747024003270780418BF9
:100FD00005C737177A0013070720B307F7021CC1AC
:100FE00021D61C41858381B701466DBF0546B547B3
:100FF000D1BF0146BD47F9B737173D00130707902A
:10100000E9BFB7150240D8559316F700D85563DFEE
:10101000060411833D8B9306170037177A001307D8
:1010200007203357D70218C1D455A182BD8A8DE25B
:1010300095463307D702058318C137170240585722
:1010400014413D8B050733D7E60218C1184171B72B
:1010500085456394B600E546E9BFBD456396B60095
:10106000D1463387E602C9BF8906E5BF3D8B9306AB
:10107000170037177A00130707203357D702F1B745
:1010800099C5371702405C4B5D8D48CB8280B717FE
:101090000240D84B1345F5FF798DC8CB828099C5A6
:1010A000371702401C4F5D8D08CF8280B717024072
:1010B000984F1345F5FF798D88CF828099C53717F2
:1010C00002405C4F5D8D48CF8280B7170240D84FF9
:1010D0001345F5FF798DC8CF828099C53717024037
:1010E0005C475D8D48C78280B7170240D8471345DB
:1010F000F5FF798DC8C78280EFF2EFC11629F57729
:10110000FD17F58FF621DA257971D58F1EA95625A1
:10111000FD779387379FF58FD6212A842EC6D58FEA
:101120009625D58FB625D58F5EA55E29C207C183CA
:1011300093F7F7CFD98F5EA96808C13BB747014045
:1011400093870780B245631EF402A2576547B387B1
:10115000E7029841930640060A07B3D7E70233D760
:10116000D702B3F7D7021207920793872703B3D7A3
:10117000D702BD8BD98FC207C1831EA445616FF012
:10118000CFBB9257E1B791C55E250967D98F5EA5A0
:1011900082805A25F977FD17F98FD5BF13F7F50F20
:1011A00085471583B395B7006319F7009307C5000A
:1011B000984301CED98D8CC382808946930745011F
:1011C000E318D7FE93070501E5B793C5F5FFF98D41
:1011D000DDB793F5F51F4EA182804A211375F51FE7
:1011E00082800A216D8D3335A000828013F7F50FC0
:1011F00085461583B397B6006311D7025A25F98F38
:101200001A2101454207418381CB0545A181B315D0
:10121000B5006D8F3335E000828089466314D700B6
:101220001A29F1BF5A29E1BFB70700209387C71ACF
:101230009843636FA702D043B386C7006316D500F7
:1012400054413E85B296D4C35041B306C500631CD9
:10125000D700B706002083A646196306D70054437B
:101260001843B29654C118C16303F50088C3828045
:10127000BA877DBFEFF28FA841112AC6EF00F03682
:10128000B706002083A74619370600209386461923
:10129000130686193245A1EF37070020930707266A
:1012A00093F5F7001307072681C51387F700419BC5
:1012B000B70500209385C51A23A2050098C18D6546
:1012C000C115AE97C19B23A2070023A00700B385D9
:1012D000E7409CC21CC3B707002023A0B71AB7077A
:1012E000002023AEB718B70700804CC31CC2032AE6
:1012F0000600B377AA0085E39307F5FF3957636CBF
:10130000F7009307050113F7F70041C313F707FF31
:10131000410763EBE706814489A022872E8461A000
:1013200058C15CC011375840B70600209386061A92
:101330009042B307E94023A0F90063F3C7009CC2C1
:10134000B70700203367EA009387471A58C09843CD
:10135000C10423200400050798C3EF00504593F70C
:10136000F400D1CBA167938707807390073037567D
:101370000000375500001306862E93050011130553
:101380000531EF20704D01A0BA87370700200329EF
:10139000C7199309C719E360F9F837070020032438
:1013A000C71A1307C71A50406374F6000C40B5F50E
:1013B0009442E38286F61440044314C33307F64094
:1013C00093060002E3F1E6F63305F4009376F500A8
:1013D000A1DAA16793870780739007303756000022
:1013E000375500001306862E9305F00C13050531C2
:1013F000EF20904601A0268541016FF06F9355C103
:10140000EFF26F91B7070020032745FF83A78719E5
:101410002A84B376F7009DE2A167938707807390D3
:10142000073037560000375500001306862E930507
:10143000401213050531EF20304201A0832605FF3D
:101440009DC2A167938707807390073037560000CD
:10145000375500001306862E9305501213050531EB
:10146000EF20903F01A093C7F7FFF98F232AF5FEE5
:10147000EF00B017B70700209387C71994430327DD
:1014800044FF130504FF369798C3793BB707002044
:101490009387871A9843050798C3EF0050316FF080
:1014A000CF898280B7E700E041572387E740238652
:1014B000E740B7F700E023A0070023A2070081461A
:1014C00094C70147D8C7370700208325071713079C
:1014D000401F814633D6E5023D4790CBD4CB98C31D
:1014E0008280EFF24F83411102C6F32750303EC68F
:1014F000B2470D478D8B6384E702A167938707800E
:1015000073900730375600003755000013064633F6
:101510009305600B13050531EF20103401A0B78748
:10152000002093870700BD8B9DC3A1679387078029
:1015300073900730375600003755000013064633C6
:101540009305B00B13050531EF20103101A0993F31
:10155000B7E700E0056723A0E710116723A0E710B5
:1015600023A40180EFE0DFD9014541016FE0FFFCDA
:1015700073110134A1679387078073900730B7F721
:1015800000E023A20700EF00F00711C5B7E700E075
:10159000116723A0E720A16793878788739007309E
:1015A0007311013473002030A16793870780739013
:1015B0000730938781809843050798C382801387FB
:1015C00081801C438DE7EFE21FF5A16793870780B9
:1015D0007390073037560000375500001306463326
:1015E0009305201013050531EF20102701A0FD17EA
:1015F0001CC391E7A1679387878873900730828027
:10160000930785007D575CC118C55CC51CC92320A4
:10161000050082802328050082809841FD569307AB
:101620008500631ED7001C49D843D8C10CC79CC590
:10163000CCC31C4188C985071CC18280B687D443AE
:101640009042E37DC7FECDB7544118451C4998C66A
:1016500054C3D4436393A600D8C3984323280500FA
:101660007D1798C388438280EFE2FFEA41112AC6C2
:10167000253F3245005DA1371335140041016FE06D
:10168000DFEB304115C2EFE21FE958451445AA8748
:10169000329758C56364D700184158C52E85CC478A
:1016A000EF2070106FE07FE98280EFE2DFE62A84AE
:1016B000E53D8344540413094402E204E184634594
:1016C0009002FD57A302F404DD3DF93D8344440438
:1016D00013090401E204E18463449002FD572302EC
:1016E000F404F13D6FE07FE55C50E1DF4A85EF00F7
:1016F000103E19C1EF00505AFD14E204E184C1B755
:101700001C48E9DF4A85EF00903C19C1EF00D05832
:10171000FD14E204E184C9B7EFE2FFDF41111DE1EE
:10172000A1679387078073900730375600003755BD
:1017300000001306C6359305001113050531EF208F
:10174000B01101A05C5D2EC62A84BDC33841B3B779
:10175000E702B9EF913D3040585C1440232C04025D
:10176000B307E602B24554C03387F600918FB697AF
:101770005CC4FD572302F40418C4A302F40495E1E9
:101780001C4899CB13050401EF00703411C5B7E76D
:1017900000E0116723A0E7201D35054541016FE0FA
:1017A000DFD913050401A93D13054402913DEDB7AE
:1017B000A16793870780739007303756000037552D
:1017C00000001306C6359305501413050531EF20AC
:1017D000B00801A0EFE23FD4411121C1B3B7A50287
:1017E000AA8485EF3305B502930770FB63E7A70270
:1017F000130585042EC6BD3C2A8401CDB245AA87B7
:1018000099C1930785042CC01CC044DC8545228502
:101810002137228541016FE05FD2A167938707805E
:101820007390073037560000375500001306C63551
:101830009305601C13050531EF20100201A0EFE2B3
:101840001FCB011132C61DE1A167938707807390FA
:10185000073037560000375500001306C63593058C
:10186000105513050531EF20207F01A02A84AE8991
:101870008DE53C419DC3A167938707807390073036
:1018800037560000375500001306C63593055055EE
:1018900013050531EF20407C01A0EF00B04015E5B5
:1018A000B247014985C7A1679387078073900730C6
:1018B00037560000375500001306C6359305A0556E
:1018C00013050531EF20407901A001497D5A930AA3
:1018D000440237EB00E0916B95A0B24781E7C53138
:1018E000014559A0631509002808EF00102DC139E2
:1018F000ED295D3983474404E207E187639447019A
:101900002302040483475404E207E18763944701F8
:10191000A30204046D316C002808EF00702B21ED48
:101920002285993329C5B2455685EF00700E228570
:10193000AD3BB52D19E123207B210549B531045C70
:10194000C9DCCE852285FD142D3B04DC1C4899CBD7
:1019500013050401EF00B01711C5B7E700E01167E8
:1019600023A0E720A939054505616FE0DFBB22858B
:101970002D3B352DD9B722850D3B152D2285ED3117
:101980004DDDB9BF15E5EFE21FB9A1679387078069
:1019900073900730375600008565375500001306F1
:1019A000C635938585AC13050531EF20E06A01A0AB
:1019B0009DCD373600209306062681470147130642
:1019C0000626214883A846006398A800931737008D
:1019D000B2978CC3C8C321A891E783A8060063937C
:1019E0000800B6870507A106E31E07FDFDF3828008
:1019F000EFE27FB241112A842EC632C47536834786
:101A000044047D572246E207E187B2456394E7002C
:101A100023020404834754047D57E207E18763945B
:101A2000E700A302040432C62EC4513E1C5CA2454A
:101A3000324689E713054402EF0010022285B531D2
:101A400041016FE09FAF370700201307871B1C433E
:101A50009443B70700209387871D81E67D5798C37D
:101A60008280184358471843DDBFEFE23FA937098A
:101A70000020B70700209304491B83A9871E2A84EE
:101A80009C4088404111A388070411052EC66D3E75
:101A90007D579307491BB245631CE40295C9B737CC
:101AA0000020938787409440D84398C610479440BD
:101AB000D0C694401047910654C29440910614C772
:101AC00098405CCB9843050798C341016FE05FA63F
:101AD00098434E9440C3637A3401370700200325AE
:101AE000C71B8C439105153ECDB737070020032552
:101AF000871B8C4391051536B70700209387871DF8
:101B00009843E374E4FC80C3C9B7EFE23F9F3734E6
:101B10000020B70900201304C441370A0020938431
:101B2000491C9C40EDDF49345C4403A9C700130500
:101B30004900193E13070A1C1C43FD171CC39C4097
:101B4000FD179CC0AD3C03250903EFF05F8B4A8570
:101B5000EFF0FF8AE9B7EFE29F9913192600AA8AEE
:101B60004A852E8A368BBA8BBE89EFF0AFF01DC145
:101B7000AA8413054005EFF0EFEF2A8409C904D9C0
:101B80008147C146631A0A00230A050225A026855B
:101B9000EFF0FF867D5565A23307FA0003070700C3
:101BA0003306F400230AE60201C78507E396D7FE51
:101BB000A3010404B94763F47703A16793870780FF
:101BC000739007303756000037550000130606376C
:101BD0009305703913050531EF20004801A0130A61
:101BE000440052852326740323227405232404040D
:101BF000EFF05FA213058401EFF0DFA13D4713056D
:101C0000C9FF33077741269500C818CC40D023067A
:101C10000404A306040423070404A30704042308FC
:101C20000404A30804045A86D6854199EFE04FFDC9
:101C300008C06384090023A08900EFF0FF96B7076E
:101C400000209387071C9843B7040020B739002071
:101C5000050798C31387441B18439384441B1389B7
:101C6000092A6310070E80C0984385476316F7065C
:101C70009389092A930AC9124E85D109EFF05F981A
:101C8000E39C3AFF37350020930AC53C1305C53C59
:101C9000EFF01F97373500209309053E1305053EE9
:101CA000EFF01F96373500201305453FEFF05F95A5
:101CB000373500201305C541EFF09F9437350020DC
:101CC00013058540EFF0DF93B707002023AC571BC7
:101CD000B707002023AE371BB70700209387C71C28
:101CE0009843050798C3370700201307071D5C5466
:101CF000144363F3F6001CC35147B387E702CA9746
:101D0000D843144718C454C4144723A246012324BB
:101D1000470198435CC8050798C3EFF05F8AB7078F
:101D2000002083A7471E054599CB9C40D8575C549B
:101D30006377F700B7E700E0116723A0E7206FE0C3
:101D40008FFEB707002083A7471ED9F79C40D857BE
:101D50005C54E3E3E7F880C041B7EFE2CFFBB7079D
:101D60000020B7550000372500009387471D014725
:101D7000814613060010938545381305A5B0E13B55
:101D80000544631E8502EF00D020631A8502A16717
:101D90009387078073900730B70700207D5723ACE7
:101DA000E71CB707002023A2A71EB707002023A423
:101DB000071EEFF00FF383A7C1806FE00FF8FD5708
:101DC000E31BF5FEA16793870780739007303756B2
:101DD0000000856537550000130606379385058496
:101DE00013050531EF20402701A0B7070020938796
:101DF000871C9843050798C38280B707002003A576
:101E0000871E8280B707002083A7871C6398071866
:101E1000EFE26FF0B70700209387871E8043050429
:101E200080C339E8B70700209387871B984318437E
:101E300005C7A16793870780739007303756000066
:101E400085653755000013060637938575AC130575
:101E50000531EF20602001A0370700201307C71BC2
:101E60009443104390C3B707002014C39387C71D42
:101E70009843050798C3C13E370600209307861D87
:101E80009C4337370020B70500201306861D130733
:101E9000072A9385451B01456375F4029C41D14691
:101EA000DC57B387D7023E971843854763F3E700B3
:101EB0000545B707002083A7C71E91C305456FE0FE
:101EC000CFE7370E0020B70E0020514F93078E1B2F
:101ED0009443944281E6FD571CC2C9B79C43DC473A
:101EE000DC47D4436374D40014C24DBF83A8870079
:101EF00003A8C700D44B1383470023A4080123225F
:101F0000180183A846006394680023A2060103A871
:101F1000060023AA07007D1823A00601945795CA3E
:101F200003A8C70183A8070283AF46002324180132
:101F300083A8070223A208011388870163940F0175
:101F400023A2160103A8060023A407027D1823A0DC
:101F5000060193860E1D03A8C70283A8060063F43A
:101F6000080123A00601B306E803BA9683A8460039
:101F700083AF880023A4170123A6F70183AF88004D
:101F800023A26F0023A46800D4CB9C4285079CC287
:101F90009C41DC57E36CF8F205450DBFB707002004
:101FA0009387071E98430145050798C38280EFE297
:101FB000EFD4370400201304841C1C40411185E732
:101FC000A1679387078073900730375600008565B7
:101FD00037550000130606379385358B13050531F9
:101FE000EF20800701A0EFF02FDC1C40FD171CC084
:101FF0001C4089CB01452AC6EFF06FDC3245410118
:102000006FE00FD3B707002083A7071CE5D7B736CB
:1020100000203735002081479386463F370F002048
:102020001305052AD14837030020370E0020854EBE
:1020300059A8DC46DC47CC4F9053985790C503A86D
:1020400007022322B8000328470093858701631302
:10205000B80050C3104323A407027D1610C38C4759
:10206000D047D84B1388470090C54CC24C4363936C
:10207000050150C3104323AA07007D1610C31307A0
:102080000F1DD0570C4363F3C50010C3330716036D
:102090002A974C4383AF85008CC723A6F70183AFF3
:1020A000850023A20F0123A405010C43D8CB85058D
:1020B0000CC31307431B184358576366E600130706
:1020C000CE1E2320D70198422DF799C3EFF0BF977A
:1020D000B70700201387071E04431384071E91CC03
:1020E000370900208549393B09C59307C91E23A03C
:1020F0003701FD14EDF823200400B707002083A763
:10210000C71EE38907EEB7E700E0116723A0E720C9
:102110000545D5B519E5B7E700E0116723A0E7202D
:102120008280EFE24FBFB707002083A7871C4111D1
:102130009DC3A167938707807390073037560000CF
:1021400037550000130606379305905413050531E3
:10215000EF10907001A02AC6493932458145EFF051
:10216000DF90B13511E5B7E700E0116723A0E72064
:1021700041016FE08FBCB707002003A7871CB7079A
:1021800000209387C71E01C7054798C3828023A0FC
:102190000700B70700201387071D18431386071D84
:1021A000B73700209387072A5148B3060703B38542
:1021B000D700884115C5C841A106BE964841C8C18F
:1021C0006314D5005441D4C1D146B306D702B697A3
:1021D000DC43D447B707002023AAD71A18C282804D
:1021E00015E7EFE24FB3A16793870780739007303D
:1021F000375600008565375500001306063793856E
:1022000025C013050531EF10306501A07D1771BFA2
:10221000EFE26FB005E5A167938707807390073001
:10222000375600008565375500001306063793853D
:10223000C5C113050531EF10306201A0B7070020BA
:102240002E8483A5471BE105EFF02FBD8545228530
:10225000EFF0BF816FE06FAEEFE2EFAB2A8705E5ED
:10226000A167938707807390073037560000856514
:102270003755000013060637938525C5130505312C
:10228000EF10905D01A0B70700209387471B5443D0
:102290002E858C4303A88600D4CD8C4323A0050350
:1022A00003A807008C46610823A2050103A80700C4
:1022B0009C43610823A4060198D71C4385071CC3CF
:1022C00011C27D55B285EFF04FFA6FE00FA75C4564
:1022D000DC4795E7EFE22FA4A1679387078073900F
:1022E000073037560000856537550000130606375E
:1022F000938525C813050531EF10105601A0D04F66
:10230000945398579385870114C6D0C250436313E2
:10231000B60054C3144323A40702FD1614C33707A1
:1023200000200327871CD45725EF8C47D047D84B74
:1023300090C5D04748434CC2938547006313B5000E
:1023400050C3104323AA07007D1610C3370700208F
:102350001307071D10436373D60014C35147338618
:10236000E602373700201307072A32975043084602
:1023700090C7C8C708464CC10CC6D8CB1C43014502
:1023800085071CC3B707002083A7471BDC5763F8EA
:10239000D700B7070020054723A6E71E0545828022
:1023A000373700201307473F50430846D0CF88D324
:1023B00008464CC10CC698D7D1B7B707002083A7F1
:1023C000C71D1CC1B707002083A7871E5CC1828080
:1023D000EFE26F94411105E5A16793870780739041
:1023E000073037560000856537550000130606375D
:1023F0009385D5CF13050531EF10104601A085E573
:10240000A167938707807390073037560000856572
:1024100037550000130606379385E5CF13050531C0
:10242000EF10904301A02EC62AC4EFF0EF973707B4
:102430000020B70700201307471B83A6871E1C43F5
:102440002245B24583C7170599CB1C43A3880704CF
:102450000544EFF0CF96228541016FE00F8E9C413D
:102460007D570144E387E7FE370600200326C61D9B
:102470000328050058416307C80063E5E60023A070
:102480000500F9B73386E640E37BF6FE958FBA97F1
:102490009CC12537014475BFB7070020054723A617
:1024A000E71E8280B707002083A7471E054581CB22
:1024B000B707002003A5871C133515000605828089
:1024C000EFE26F8537040020EFF00F8E1304C41F76
:1024D0001C40B1E7373500201309054313050543B8
:1024E000EFF00F923735002093044544130545441F
:1024F000EFF00F91B707002023A8271F0146B70769
:102500000020C145114523AA971EEFF0AFAC08C0CB
:1025100019C5B75500009385053BEFF0AFC6EFF046
:102520000F8A6FE08F81EFD21FFF4CC108C9AA87C5
:102530006362B602184D158E0545637BE6009385F0
:102540004700B707002003A5471FEFF00F8D014597
:102550006FD0BFFE6375D6000545E3FBD5FE9385BE
:102560004700B707002003A5071FC5B7EFD2BFFA82
:102570002A84AE8432890C4CA6864A86A69522858A
:102580005D3719E16FD07FFB1C4C2285BE941C5037
:102590008297D5B7EFD23FF8B707002083A7071F70
:1025A0004111AA84DC472EC6C04713054400EFF052
:1025B000AF8983474402324613F7470011CBA68503
:1025C00022856D371C502285829741016FD0FFF61E
:1025D000F99B2302F402FDB7EFD2FFF3370400208A
:1025E0009306041F98421C4391EBB7070020938782
:1025F000471F904398C390C26FD03FF45C47FD558E
:102600008843493FF1BFEFD29FEE15694111B70AE8
:102610000020B7090020370B0020B70B002013095A
:10262000C93883A70A1F984329CBDC47814C03ACE8
:102630000700EFF08FFBEFF04FFC83A7891F2A8480
:102640009384891F130ACB1F636CF50288C0638FC4
:102650000C0283A74B1F90431336160003250A0074
:10266000B3058C40EFF0CFB8EFF07F9411EDB7E7F2
:1026700000E0116723A0E72001A8854C014C55BF5D
:10268000A13F80C0EFF0BF92214C05A00146E36757
:1026900085FDEFF0DF91A2856285ED3DF5B79247AC
:1026A000B2458297824763DD070003250A00014691
:1026B0008A85EFF0CF9835D582472245E3C107FEE2
:1026C00022445C4895E3EFF04FF39C40AA8C63737F
:1026D000F5001937824723A09401FD17E367FCFC3E
:1026E0008A07CA979C43828713054400EFE0DFF511
:1026F000D9BF834744020C4C924693E7170023024C
:10270000F4026686B6952285393D45D18347440259
:1027100013F7470019CB1C4C924566862285BE955F
:10272000B1351C502285829749B7F99B2302F402E8
:10273000CDBF83474402F99B2302F402BDB7834710
:102740004402924593E717002302F4020CCC9DE16A
:10275000A16793870780739007303756000037557D
:1027600000001306863B9305903513050531EF10E5
:10277000B00E01A0E6866686E69522856D3335B7F4
:102780008347440213F727005DF72285EFE03FC738
:1027900029BFEFD25FD82D33B707002083A7C71F0B
:1027A0009DE3A16793870780739007303756000039
:1027B000375500001306863B93059011130505312C
:1027C000EF10900901A0B7070020B755000037258A
:1027D0000000938707203947814613060010938530
:1027E000053D13056560EFF00FB745DD6FD0FFD4F1
:1027F000B707002083A7071737177A0013070720AA
:10280000B3D7E7023707002093F7F70F2303F7202A
:102810001307803EB387E702370700202312F72013
:102820008280EFD25FCF2A841165011185451105A1
:10283000EFE0FF86930700207C82371501408D472B
:102840003EC44C00E147130505803EC6EFE06FD85B
:1028500022C837440140B70708000C08130504805C
:102860003ECC02CA231E0100EFE01F8985451305F7
:102870000480EFE05F9105616FD03FCCEFD21FC8BD
:10288000B7440140AE893289014493840480634592
:1028900024014A856FD0DFC9930500042685EFE047
:1028A0005F947DD9B3878900838507002685050459
:1028B000C205C181EFE0FF91D9BF138701811C439D
:1028C000B74600209386C6853E95636BD500B786D4
:1028D00000209386068063E5A60008C33E858280BB
:1028E000FD57EDBF232605000CC150C12324050070
:1028F000054582805C45544118458507B3E7D702FA
:10290000638EE70058451C41BA978CA35C4558413B
:102910008507B3E7E7025CC505458280795582806B
:10292000EFD27FBF79711306000281450808EFD00E
:102930009FC18545114502C202C402C6EFE02FF6D1
:10294000854513050020EFE08FF51165EFE0CFDA44
:10295000371401408547130504804C007C8202C671
:10296000EFE02FC7C147130504804C007C8202C6EC
:10297000EFE02FC6930700024C00130504807C8211
:102980003724014002C6EFE0CFC413050440EFD066
:102990003FF985473ECA3ECCB7070E003ECE0C0835
:1029A0008D47130504402302F10202C802D0EFD084
:1029B0001FFB854513050440EFE0CF8085451305D7
:1029C0000440EFD03FFF814513050440EFE0EF8F57
:1029D00013050440EFE02F80930404402685EFE0C8
:1029E0002F806DFD1305044037240140EFD0DFFF39
:1029F000930404402685EFD0DFFF6DFD13050440EE
:102A0000EFE02F8EB70700202394A72045616FD0F9
:102A1000DFB2EFD25FB079711306C0028145480082
:102A2000EFD07FB285450545EFE08FE537040240E2
:102A300013058400EFE06F9EB72701409387C744DA
:102A40003EC2B70700209387C7203EC48D473EC8CB
:102A5000930700083ECC930700103ECE930700403A
:102A60003ED0930700023ED24C008D6713058400D0
:102A70003ED402C602CA02D6EFE0EFB045616FD085
:102A8000DFABEFD25FA9370502408545210537242A
:102A90000140EFE0CFB2130504409D460546814555
:102AA000EFD03FF7130504409D4609469145EFD00E
:102AB0005FF69D460D46130504409545EFD07FF522
:102AC000130504408545EFD0FFEF8545130504400D
:102AD000EFD0BFF26FD07FA6EFD2FFA341118545A3
:102AE00013050004EFE0AFDBA147372401407C82EF
:102AF00085473EC44C00C147130504803EC6EFE045
:102B00004FAD014613050480A145EFE08FB8914712
:102B10004C00130504807C82EFE0AFAB0146130547
:102B200004809145EFE0EFB6930700084C001305D1
:102B300004807C82EFE0EFA9014613050480930531
:102B40000008EFE00FB5930700104C001305048058
:102B50007C82EFE00FA80146130504809305001066
:102B6000EFE02FB3930700204C00130504807C8214
:102B7000EFE02FA601461305048093050020EFE047
:102B80004FB1930700404C00130504807C82EFE0B6
:102B90004FA401461305048093050040EFE06FAF9A
:102BA0008567938707804C00130504807C828564C9
:102BB000EFE02FA201469385048013050480EFE027
:102BC0004FAD4C00130504806482EFE08FA00146F6
:102BD000130504808565EFE0CFAB89644C001305D5
:102BE00004806482EFE0EF9E01461305048089654E
:102BF000EFE02FAA91674C00130504807C82EFE080
:102C00004F9D0146130504809165EFE08FA8E177A1
:102C10004C00130504807C82EFE0AF9B0146130556
:102C20000480A165EFE0EFA64C00371501406482F7
:102C3000EFE02F9A0546896537150140EFE06FA553
:102C400041016FD09F8FEFD21F8DEFE08FA46FD027
:102C5000DF8EEFD25F8C79712A89854513050004D8
:102C6000EFE0EFC337240140930700028D44FC825C
:102C70004C08C147130504803ECE26CCEFE06F958B
:102C800001461305048093050002EFE08FA08545FF
:102C90004145EFE0CFC0854513050004EFE00FC2CA
:102CA0008547FC824C08E1473715014026CC3ECED3
:102CB000EFE02F928947FC824C089147371501407D
:102CC000372400403ECEEFE0CF900C10B7070C0049
:102CD000130504804AD03ED402D223160102EFE04D
:102CE000AFC1930770357C86680085473EC844872E
:102CF000EFE06F9B05461305048093055052EFE00B
:102D0000EFC9854513050480EFE0EFC745616FD03B
:102D1000DF82EFD25F8079712A898545130500042F
:102D2000EFE0EFB737240140930700048D44FC82A5
:102D30004C08C147130504803ECE26CCEFE06F89D6
:102D400001461305048093050004EFE08F94854548
:102D50004145EFE0CFB4854513050008EFE00FB61D
:102D60009147FC824C08E1473715014026CC3ECE06
:102D7000EFE02F86A147FC824C08914737150140B0
:102D8000372400403ECEEFE0CF840C10B7070C0094
:102D9000130504C04AD03ED402D223160102EFE04C
:102DA000AFB5930780357C86680085473EC8448769
:102DB000EFE06F8F0546130504C093055052EFE016
:102DC000EFBD8545130504C0EFE0EFBB45616FD053
:102DD000CFF6EFD24FF479712A8985451145EFE09E
:102DE0000FAC3714014089478D44FC824C08C14721
:102DF000130504803ECE26CCEFD0BFFD014613055F
:102E000004808945EFE0EF8885451145EFE02FA963
:102E1000854537050200EFE06FAA9147FC824C0818
:102E2000E1471305048026CC3ECEEFD09FFAA147A0
:102E3000FC824C089147130504803ECE3744004085
:102E4000EFD03FF90C10B7070C00130504404AD02F
:102E50003ED402D223160102EFE00FAA930760339B
:102E60007C86680085473EC84487EFE0CF830546EF
:102E70001305044093055052EFE04FB2854513050A
:102E80000440EFE04FB045616FD02FEBEFD20FE77A
:102E90007971AA8985452145EFE06FA03719014076
:102EA00085470D44C1444C08130509C0FC8226CE59
:102EB00022CCEFD01FF20146130509C08545EFD0A3
:102EC0005FFD85454145EFE08F9D85451305001069
:102ED000EFE0CF9EE1474C0837150140E48222CC59
:102EE0003ECEEFD01FEF93070002FC824C089147C3
:102EF000371501403ECEEFD0DFED0C10B7070C00C8
:102F0000372500404ED03ED402D223160102EFE016
:102F1000AF9E930790357C86680085473EC8408702
:102F2000EFD07FF805469305505237250040EFE07B
:102F3000EFA6854537250040EFE0EFA445616FD04F
:102F40002FDFEFD24FDD3714014013050440014657
:102F500093050020EFD0FFF31305044001469305CD
:102F60000040EFD01FF3856501469385058013056A
:102F70000440EFD01FF26FD04FDCEFD22FD8797121
:102F80002A8A854513050002EFE06F91371401404E
:102F900093070010FC820D49C1474C0813050480BB
:102FA0003ECE4ACCEFD0FFE2014613050440930524
:102FB0000010EFD01FEE930700204C08130504808B
:102FC000FC82EFD01FE1930900404C0813050480F8
:102FD000231A31018564EFD0DFDF4C08130504802C
:102FE00093840480E482EFD0DFDEA13F8545214554
:102FF000EFE0EF8A854537050400EFE02F8CE147CD
:103000004C08130504C0231A31014ACC3ECEEFD040
:103010005FDC91474C08130504C0E482375400403C
:103020003ECEEFD01FDB0C10B7070C001305048059
:1030300052D03ED402D223160102EFE0EF8B930769
:1030400070137C8685475C87680085473EC8EFD053
:103050009FE505461305048093055052EFE00F9459
:10306000854513050480EFE00F9245616FD04FCC8A
:10307000EFD26FCA7971AA8485454145EFE02F826E
:10308000854513050002EFE08F8185453705100067
:10309000EFE0CF8285670D44FC824C08E14737158D
:1030A000014022CC3ECEEFD0DFD291473715014010
:1030B000FC824C089147130505403ECEEFD07FD1EE
:1030C000B7070C000C10375500403ED426D002D272
:1030D00023160102EFE04F82054693055052375503
:1030E0000040EFE0AF8B930750147C866800854763
:1030F0003EC84087EFD03FDB854537550040EFE0C5
:103100008F8845616FD06FC3397106DE16DC1ADA1D
:103110001ED82AD62ED432D236D03ACE3ECC42CA8F
:1031200046C872C676C47AC27EC0F929F250E2520D
:103130005253C2533255A255125682567247E24735
:103140005248C248324EA24E124F824F2161730044
:103150002030397106DE16DC1ADA1ED82AD62ED4B3
:1031600032D236D03ACE3ECC42CA46C872C676C4B7
:103170007AC27EC01D2BF250E2525253C2533255D6
:10318000A255125682567247E2475248C248324E02
:10319000A24E124F824F216173002030397106DE3A
:1031A00016DC1ADA1ED82AD62ED432D236D03ACE2F
:1031B0003ECC42CA46C872C676C47AC27EC0412B93
:1031C000F250E2525253C2533255A2551256825611
:1031D0007247E2475248C248324EA24E124F824FC7
:1031E000216173002030397106DE16DC1ADA1ED830
:1031F0002AD62ED432D236D03ACE3ECC42CA46C897
:1032000072C676C47AC27EC0CD23F250E2525253C7
:10321000C2533255A255125682567247E24752485F
:10322000C248324EA24E124F824F216173002030AD
:10323000397106DE16DC1ADA1ED82AD62ED432D21E
:1032400036D03ACE3ECC42CA46C872C676C47AC29E
:103250007EC02D2DF250E2525253C2533255A25528
:10326000125682567247E2475248C248324EA24E28
:10327000124F824F216173002030397106DE16DC57
:103280001ADA1ED82AD62ED432D236D03ACE3ECC36
:1032900042CA46C872C676C47AC27EC0EF002069B0
:1032A000F250E2525253C2533255A2551256825630
:1032B0007247E2475248C248324EA24E124F824FE6
:1032C000216173002030B7070020039787208147D2
:1032D0002A97634F070009CD05669306F6FFB68768
:1032E0006358C700AA876305D50093170701C183F8
:1032F0003E858280EFD22FA2EFF08FE2EFF06FF1E8
:10330000EFF02FF86FD06FA3375700000327074364
:10331000B707002023AEE7203757000003274743B5
:10332000B707002023ACE720375700000327874367
:10333000B707002023AAE7208280EFD2CF9DB707EE
:1033400000200395C7204137EF00B032B7070020B7
:1033500083A5C721EF00D0026FD02F9EEFD2AF9B85
:10336000B70700200395E720B93FEF009030B7077B
:10337000002083A54721EF00B0006FD00F9CEFD253
:103380008F99B707002003950721353FEF00702E76
:10339000B707002083A58721EF00807E6FD0EF99CB
:1033A000EFD26F97B70700201387C72083D5C720B8
:1033B00056233223375500001305C53DEF00D04991
:1033C000375400009D3F8325843DEF00607BEF0074
:1033D0003024AA85375500001305053FEF00D0477C
:1033E000B53F8325843DEF00A079EF007022AA85C8
:1033F0003755000013058540EF00104649378325F7
:10340000843DEF00E077EF00B020AA85375500003B
:103410001305C541EF0050446FD02F92EFD2AF8F0C
:10342000EFF08FEB6FD06F91EFD2EF8E85472E8646
:10343000930500086307F5028947930500106302AE
:10344000F5028D4793050020630DF5009147930524
:1034500000406308F5009547631DF5008565938579
:1034600005803725014013050580EFF0CFFD6FD0B3
:10347000CF8C99478565E306F5FE9D478965E30294
:10348000F5FEA1479165E30EF5FCA547A165E30AAA
:10349000F5FCA947E31DF5FCA145E1B7EFD20F8686
:1034A000370400209307040201491304040219475A
:1034B000D4436392A60893094002B3093903330A3F
:1034C000340183470A0095E7AA841385C900229531
:1034D000EFF04FC1994703258A006390F402EFF0A3
:1034E0004FF7930740023309F902854722992300D9
:1034F000F900330534016FD0AF839D476395F40025
:10350000EFF03F81F9BF89476395F400EFF07F8CBE
:10351000C9BFA1476395F400EFF05F97D9B78D4716
:103520006395F400EFF07FA56DBF9547E39BF4FA38
:10353000EFF01FB47DB7050993874702E31AE9F658
:10354000014555BFEFC23FFDB7070020B73500204A
:1035500023AEA70C13060040938585451545EFF073
:10356000FFF3B707002023A6A7246FC01FFDB707EE
:10357000002083A787236399A700B707002083C78C
:103580000725858B3E858280B707002083A7C72348
:103590006398A700B707002083C70725898BDDB78D
:1035A000B707002083A707246398A700B707002068
:1035B00083C70725918BF9B7B707002083A7472456
:1035C0006398A700B707002083C70725A18B5DBFBD
:1035D000B707002083A787246399A700B7070020B7
:1035E00083C7072593F7070271BFB707002003A71A
:1035F000C7249307F00FE317E5F8B707002083C748
:10360000072593F70704BDBFEFC2FFF03744004022
:103610009305505213050440EFD05FBD15C9130543
:103620000440EFD09FBB9375F50FB70700202384AC
:10363000B722B707002003A507241C4D10495449A1
:103640008507B3E7C7026385D7003105EFF08FAA7E
:10365000374400409305707213050440EFD01FB942
:103660001DC5B707002083A707249633BA3363E24A
:10367000E60201469305707213050440EFD01FB2B5
:10368000B70700209387072598236D9B98A36FC0E9
:10369000DFEAD84F1386160092B3B307D7008C2306
:1036A00013050440EFD0FFB2DDB7EFC2DFE63754B9
:1036B00000409305505213050480EFD03FB315C965
:1036C00013050480EFD07FB19375F50FB707002085
:1036D0002388B722B707002003A587241C4D104973
:1036E00054498507B3E7C7026385D7003105EFF07A
:1036F0006FA0375400409305707213050480EFD01B
:10370000FFAE05C9B707002083A787249633BA33D5
:1037100063E3E60201469305707213050480EFD05F
:10372000FFA7B70700209387072598231377F7FD96
:1037300098A36FC09FE0D84F1386160092B3B307CB
:10374000D7008C2313050480EFD0BFA8DDB7EFC2EC
:103750009FDC9305505237550040EFD03FA915C963
:1037600037550040EFD07FA79375F50FB7070020BE
:10377000238AB722B707002003A5C7241C4D104990
:1037800054498507B3E7C7026385D7003105EFF0D9
:103790006F969305707237550040EFD03FA505C96D
:1037A000B707002083A7C7249633BA3363E3E60242
:1037B00001469305707237550040EFD03F9EB70722
:1037C00000209387072598231377F7FB98A36FC0F2
:1037D000DFD6D84F1386160092B3B307D7008C23D9
:1037E00037550040EFD0FF9EDDB7EFC2DFD2372460
:1037F00000409305505213050480EFD03F9F15C938
:1038000013050480EFD07F9D9375F50FB707002057
:103810002380B722B707002003A587231C4D10493A
:1038200054498507B3E7C7026385D7003105EFF038
:103830006F8C372400409305707213050480EFD01D
:10384000FF9A1DC5B707002083A787239633BA3395
:1038500063E2E60201469305707213050480EFD01F
:10386000FF93B7070020938707259823799B98A398
:103870006FC0BFCCD84F1386160092B3B307D700E2
:103880008C2313050480EFD0DF94DDB7EFC2BFC8EF
:103890003724004093055052130504C0EFD01F9504
:1038A00015C9130504C0EFD05F939375F50FB707E3
:1038B00000202382B722B707002003A5C7231C4D91
:1038C000104954498507B3E7C7026385D70031051E
:1038D000EFF04F823724004093057072130504C047
:1038E000EFD0DF901DC5B707002083A7C72396330D
:1038F000BA3363E2E602014693057072130504C011
:10390000EFD0DF89B7070020938707259823759BA1
:1039100098A36FC09FC2D84F1386160092B3B30707
:10392000D7008C23130504C0EFD0BF8ADDB7EFC2E8
:103930009FBE9305505237250040EFD03F8B15C9ED
:1039400037250040EFD07F899375F50FB70700202A
:103950002386B722B707002003A547241C4D104932
:1039600054498507B3E7C7026385D7003105EFE007
:103970007FF89305707237250040EFD03F871DC553
:10398000B707002083A747249633BA3363E2E602E1
:1039900001469305707237250040EFD03F80B7078E
:1039A00000209387072598235D9B98A36FC0FFB8DD
:1039B000D84F1386160092B3B307D7008C23372550
:1039C0000040EFD01F81DDB7EFC2FFB441112A8460
:1039D0002EC632C4EFF0BFB92A8935E9B245224676
:1039E000B707002083A487234CCC2310040232B0F5
:1039F00063958402054693057072372400401305D1
:103A00000480EFD0AFF99A30DC4C130504809306A4
:103A1000170096B0BA978C230DA8B707002083A48F
:103A2000C723639A840237240040930570721305FC
:103A300004C00546EFD08FF69A30DC4C130504C065
:103A40009306170096B0BA978C23EFD08FF84A856B
:103A500041016FC09FAEB707002083A40724639580
:103A600084023744004093057072130504400546F4
:103A7000EFD0CFF29A30DC4C1305044093061700C8
:103A800096B0BA978C23D1B7B707002083A44724F8
:103A90006393840293057072372500400546EFD08A
:103AA000EFEF9A30DC4C372500409306170096B0B4
:103AB000BA978C2359BFB707002083A48724639843
:103AC0008400054693057072375400400DBFB70758
:103AD000002083A4C724E39C84F6930570723755B5
:103AE00000400546EFD08FEB9A30DC4C3755004054
:103AF0009306170096B0BA978C2381BFEFC2BFA17F
:103B000085452945EFF05F92B7040020EFF0CFFF25
:103B100037040020EFF0DF880546930570723755B3
:103B20000040EFD0AFE70325C42431469385840FCE
:103B3000EFF09FE91305803EEFE0CFDDE1BFEFC27C
:103B40009F9D716513050520EFF0DF9FEFF01F8D3E
:103B5000EFF04FFAB7070020B755000037450000D7
:103B60009387472515478146130600109385C54363
:103B70001305C5AFEFD03FFEEFE02F9E6FC0FF9B58
:103B8000797122D4135475014ECE52CC93199500FD
:103B900006D626D24AD056CA5AC81374F40F93D9FF
:103BA0009900135AF50169C49307F00F6308F40EE6
:103BB0009397390037070004B3E9E700130414F8BA
:103BC0008144014B13D77501939A95001377F70F32
:103BD00093DA9A0013D9F50145CF9307F00F630CE0
:103BE000F7028E0A130717F8B7070004B3EAFA00C2
:103BF0003A94014633452A01BD47AA86930514002D
:103C000063E0971017270000130707848A04BA940B
:103C10009C40BA9782871304F40F63960A0C93E4CE
:103C200024000946C1BF01451307F00FB707400044
:103C3000B2502254A6075E07A5837E05D98F925401
:103C40000259F249624AD24A424B5D8D45618280F7
:103C5000CA86D689328B8947630FFB088D47E304F8
:103C6000FBFC854736856310FB1A01478147C9B7BE
:103C7000639D090413D77501939A95001377F70F85
:103C800091440144054B93DA9A0013D9F50131F7B9
:103C9000639D0A0093E414000546A9BF63920902DC
:103CA000A1441304F00F094B31BF568571249307CB
:103CB000B5FF098CB39AFA001304A4F801461DBF9E
:103CC000B1441304F00F0D4BF5BD4E852EC6AD2447
:103CD0009307B5FF1304A0F8B399F900098C814448
:103CE000014BB245C5B593E434000D4621B7894771
:103CF000D286E315FBF636851307F00F81470DBF1B
:103D000041639306F3FF13D6090193D80A01B3F771
:103D1000D900B3FADA0033885703B389F80213578E
:103D20000801B30A5603D6994E97330616036373F8
:103D300057011A96C167FD17B376F7003378F8007C
:103D4000C206C2969399660093570701B3393001B2
:103D5000E982B2979A07B3E6D900B3E9D7009397FF
:103D6000490063D9070013D7190093F71900B36905
:103D7000F7002E841307F4076350E00493F77900EB
:103D800099C793F7F90091466383D70091099397F8
:103D9000490063D90700B70700F8FD17B3F9F90028
:103DA000130704089307E00F63CBE70493976900B8
:103DB000A5831377F70FADBD8547B386E74011C7DD
:103DC0006D4601478147E345D6E61307E40933977B
:103DD000E9003337E000B3D7D900D98F13F7770064
:103DE00019C713F7F70091466303D700910713979C
:103DF0005700634C07009A07A583014715BD1307B9
:103E0000F00F814735B52E84B5B7054781470DB50D
:103E100037068000135775019307F6FF1377F70FE6
:103E20009305E007B3F6A7009357F50163FCE5009F
:103E30009305D00963FAE500370500801345F5FFC7
:103E40003E9582800145828093055009D18E63CDD5
:103E5000E500130660093307E64033D7E600330573
:103E6000E040F5F33A8582801307A7F63397E60022
:103E7000FDB7411106C622C426C20DCD9357F541A8
:103E800033C4A7001D8CAA8422857D209307E009F6
:103E90003387A74093076009FD8063CCE702A14602
:103EA0009377F70F63D5A60061153314A400260499
:103EB000258021A0814481470144260413559400A4
:103EC000B2402244DE07FE045D8D458D92444101DF
:103ED00082809307900963DDE7009307B50195465B
:103EE000B317F400898E3354D400B337F0005D8CDF
:103EF000954763D6A7009307B5FF3314F400B706C0
:103F000000FCFD16937774003376D40085C3937755
:103F1000F4009145638CB70011069317560063D7E0
:103F200007009307F009758E3387A74013146600C6
:103F300025809377F70F51B7C167637CF50293072C
:103F4000F00F1307000263EBA70097170000938799
:103F5000A753AA9788233305A7408280218197170A
:103F6000000093876752AA97882361473305A740CB
:103F70008280B7070001636DF5006181971700002B
:103F800093878750AA97882321473305A7408280CB
:103F90004181971700009387274FAA9788234147AD
:103FA0003305A7408280B3C7A5008D8B3307C500BA
:103FB00081E78D4763EDC700AA87637EE5089421FA
:103FC00085078505A38FD7FEE3EBE7FE8280937616
:103FD0003500AA8789CA942185078505A38FD7FE56
:103FE00093F63700C5BF9376C7FF138606FE63F0CE
:103FF000C70683A3050083A2450083AF850003AFF6
:10400000C50083AE050103AE450103A3850183A866
:10401000C5019385450223A0770003A8C5FF23A20D
:10402000570023A4F70123A6E70123A8D70123AA59
:10403000C70123AC670023AE17019387470223AE65
:1040400007FF75B790419107910523AEC7FEE3EBDB
:10405000D7FEE3E6E7F6828039713EDA2ED232D41B
:1040600036D63AD842DC46DE9387418122CC804363
:1040700026CA06CEAA8409C41C4C99E32285FD29D0
:104080000C4454102686228536C6EF001015F240E7
:104090006244D24421618280011126CA4AC806CEF8
:1040A00022CC4EC652C4AA842E8901C51C4D91E370
:1040B000F1219C4C804499E32685C9219717000083
:1040C0009387874E631BF402C0405E24A18BB1C767
:1040D0001C48A1C7FD59294A1C4483450900FD1706
:1040E000B1E91CC463DD07062286A945268569203F
:1040F000FD576308F502294535A0971700009387FF
:10410000A74C6314F4008044C9B797170000938745
:10411000A747E31CF4FAC0444DBFA2852685192A9F
:1041200055D97D55F2406244D2444249B249224AAF
:10413000056182801CC4050963D70700184C63CA57
:10414000E700638845011C401387170018C08CA343
:1041500061B7228626850D20E31035F9D9B71C40BA
:104160001387170018C0294798A371B79387418117
:10417000AA8588436FF05FF2011122CC26CA4AC893
:1041800006CE4EC6AA842E89328401C51C4D91E309
:10419000F52697170000938727416317F406C04060
:1041A0001C4C1CC45E24A18BC1C31C48B5CF1C4849
:1041B00008409379F90F1379F90F1D8D5C48634618
:1041C000F500A2852685692C25E51C440505FD170B
:1041D0001CC41C401387170018C0238037015C489B
:1041E0006388A7005E24858B81CBA9476316F900FD
:1041F000A2852685B5240DEDF24062444A85D2445D
:104200004249B24905618280971700009387C73BF6
:104210006314F400804469B7971700009387C7368A
:10422000E310F4F8C044ADBFA2852685212041D11A
:104230007D59D9B741119387418126C2844322C455
:104240004AC006C62A892E8489C49C4C99E32685D7
:1042500035269717000093872735631BF402C0406B
:104260000317C40093170701C18393F68700ADEAD3
:1042700093F6070195EEA5472320F900136707047D
:104280005AA47D55B24022449244024941018280A1
:1042900097170000938747336314F4008044C9B72D
:1042A000971700009387472EE31CF4FAC0444DBFD4
:1042B000918B9DC34C5889C9930744046384F500CE
:1042C0004A85292B232A04025E242322040093F723
:1042D000B7FD5EA41C481CC05E2493E787005EA463
:1042E0001C4899EB5E241307002093F70728638589
:1042F000E700A2854A8591295E2413F717001DC3A4
:104300005C4823240400B307F0401CCC1C48014542
:10431000B5FB8317C40013F707082DD793E70704ED
:104320005EA485B7898B014791E3584818C4F9BF4B
:10433000DE25011122CC26CA06CE4AC84EC613F786
:104340008700AA842E8479EBD841634DE000B84100
:10435000634AE0000145F2406244D2444249B24916
:104360000561828058547DD703A9040093963701D4
:1043700023A0040063DB060670485E24918B99C776
:104380005C401D8E5C5899C33C401D8E5C540C50A3
:10439000814626858297FD575A24631DF500944077
:1043A000F54763E8D706B70740208507B3D7D7009E
:1043B000858BA5C31C48232204001CC0931737011A
:1043C00063D80700FD576314F5009C4091E368C86B
:1043D0004C5823A02401BDDD930744046384F500F9
:1043E0002685ED2E232A0402B5B70C5001468546DA
:1043F00026850297FD572A86E311F5F89C40B5DF24
:1044000075476385E70059476393E70423A02401B8
:1044100091B7136707045AA47D5535BF83A90501D9
:10442000E38A09F203A905008D8B23A03501330926
:104430003941014791E3D84918C4E35D20F11C5488
:104440000C50CA864E86268582976347A0005E245C
:1044500093E707045EA4C9B7AA993309A940F1BF3D
:104460009C49A5C3011122CC06CE2A8411C51C4D3E
:1044700081E72EC62122B245971700009387C71205
:10448000639CF5004C408397C5009DC7228562441C
:10449000F24005616FF0DFE9971700009387C712BC
:1044A0006394F5000C44C5B7971700009387C70DB8
:1044B000E39BF5FC4C44C1BFF240624401450561F9
:1044C000828001458280411122C406C62A844EA5FD
:1044D00072A52320050023220500232405002322A2
:1044E000050623280500232A0500232C0500214664
:1044F00081451305C505EFC00F8597170000938709
:1045000087B45CD0971700009387A7B61CD4971781
:104510000000938787BA5CD4971700009387E7BCA5
:1045200000D01CD8B240224441018280970500008F
:10453000938545F391AA411126C213068006938400
:10454000F5FFB384C4024AC02E8922C406C69385EF
:1045500044072D2E2A8401CD232005002322250186
:10456000310508C4138684068145EFB0DFFD22853E
:10457000B240224492440249410182801C4DA5E789
:10458000411106C622C497070000938767FA1CD51D
:104590009387C1819C4323240504232605042328F3
:1045A00005046314F50085471CCD2A84352848C0CE
:1045B00022851D2808C42285052848C44840014694
:1045C0009145EFF05FF008440546A545EFF0BFEFD9
:1045D00048440946C945EFF01FEF85471CCCB2405F
:1045E000224441018280828041119387C18126C289
:1045F00084434AC006C69C4C22C42A8981E726858A
:10460000EFF0DFF7938484048044DC40FD1763D629
:1046100007009C40B9CF8440C5BF0317C40039E7E9
:10462000C1778507232204062320040023220400E7
:10463000232404005CC423280400232A0400232C20
:104640000400214681451305C405EFB0DFEF232A9E
:104650000402232C040223240404232604042285B8
:10466000B2402244924402494101828013048406EC
:1046700071BF91454A85EFF01FEC88C049FDB147F5
:104680002320F9000144E1BF797122D44AD052CCF1
:1046900056CA5AC85EC606D626D24ECE2A8AAE8AD8
:1046A000130485040149054BFD5B09ECB25022540B
:1046B0004A8592540259F249624AD24A424BB24B5D
:1046C00045618280044483294400FD1963D40900B4
:1046D0000040E1BFDE24637BFB008397E400638737
:1046E0007701A6855285829A3369A900938484064E
:1046F000E9BF1971A6DAAE848395E500A2DC86DEF7
:10470000328463DB0500DE2423A0060093F707084C
:1047100085E7930700401DA0300836C6EF007023E0
:10472000B246E34205FE7247BD67F98F7977BA97C3
:1047300093B717009CC2F1BF930700041CC0F6504A
:104740006654D654014509618280DE25011122CCD0
:1047500006CE26CA4AC8898B2E8489CF9307740453
:104760001CC01CC885475CC8F2406244D244424920
:104770000561828074003000AA84EFF09FF7A245A3
:104780002A892685212219E98317C40013F70720F7
:1047900061FFF19B93E727005EA4C9B7970700006C
:1047A000938707D99CD45E2408C008C893E70708FC
:1047B0005EA4A2475CC8B24781CF8315E40026857A
:1047C000EF00501C11C55E24F19B93E717005EA417
:1047D0005E243369F9002316240179B7DDC583A768
:1047E000C5FF411122C406C626C21384C5FF63D388
:1047F00007003E94AA84EF00B02097C7FF1F93875D
:10480000E7A59C4391EF2322040097C7FF1F23A72E
:1048100087A42244B2402685924441016F00701E55
:10482000637EF40014403307D4006396E700984396
:10483000DC43369718C05CC0C9BFBA87D84319C3D8
:10484000E37DE4FE94433386D700631F8600104067
:10485000B29694C33386D700E31DC7FA104358437A
:10486000B29694C3D8C375B76375C400B1479CC0F2
:104870004DB71040B306C4006316D7001443584325
:10488000B29614C058C0C0C369B78280011126CA4D
:1048900093843500F19806CE22CC4AC84EC6A104B6
:1048A000B14763F9F404B14463E8B4042A89EF0022
:1048B000301597C7FF1F9387679A98433A8439E466
:1048C00097C7FF1F9387C7999C4381EB81454A8512
:1048D000812797C7FF1F23A5A798A6854A850D2F77
:1048E000FD59631B3507B1472320F9004A85EF00C6
:1048F000501129A0E3DA04FAB1471CC10145F24086
:104900006244D2444249B249056182801C40858F8D
:1049100063C10704AD4663F6F6001CC03E9404C0B4
:1049200001A85C406315870217C7FF1F2328F79271
:104930004A85EF00100D1305B400930744006199F8
:104940003307F5404DDF3A94898F1CC04DBF5CC3DF
:10495000C5B722874040A5B7130435007198E3001E
:1049600085FCB305A4404A856525E31A35FBA5BF40
:104970001C46FD171CC663DA0700184E63C5E70026
:10498000A9476394F5006FF02FFF1C422E85138713
:10499000170018C28CA38280011122CC26CA4AC8F3
:1049A0004EC652C406CE2A89AE893284B304D600DC
:1049B0007D5A63149400014509A80C204E864A854F
:1049C000EFF01FFB0504E31645FFF2406244D244BA
:1049D0004249B249224A05618280357122CD26CBF7
:1049E0004AC94EC706CF52C556C35AC1DEDEE2DC05
:1049F000E6DAAA89AE843289368409C51C4D99E36A
:104A0000EFF0DFB797170000938707BA6398F40CAD
:104A100083A44900DE24A18BE5C79C48F5C3930716
:104A20000002A304F1029307000302D22305F1025E
:104A300022C6930B5002971A0000938AEABA054CDB
:104A4000294B4A841C2099C3639F770DB30C2441E2
:104A5000638E0C00E6864A86A6854E85EFF0DFF36E
:104A6000FD57630FF51C9256E69636D21C206389DB
:104A7000071CFD571309140002C802CE3ECA02CC1F
:104A8000A309010482D48345090015465685A92F40
:104A900013041900C24751E913F7070109C71307A7
:104AA0000002A309E10413F7870009C71307B00246
:104AB000A309E104834609001307A002638FE606F9
:104AC000F2474A84814625461820930514001307AF
:104AD00007FD6377E60AB5CA3ECE85A897170000A2
:104AE000938787AE6395F40083A4890025B7971751
:104AF0000000938767A9E39FF4F083A4C90019BF5E
:104B0000A6854E85EFF00FF319D97D55FA406A441A
:104B1000DA444A49BA492A4A9A4A0A4BF65B665C21
:104B2000D65C0D618280050431BF330555413315D4
:104B3000AC00C98F3EC82289B9B7324793064700F7
:104B4000184336C6634707023ACE18209307E0029F
:104B5000631DF70418309307A002631BF702B247E6
:104B60000904138747009C433AC663C107023ECA43
:104B70002DA83307E04093E727003ACE3EC8F1B7AF
:104B8000B387670385462E84BA973DBFFD57C5B7E7
:104B9000050402CA81468147254618209305140062
:104BA000130707FD6374E606F9F20C200D4617158E
:104BB00000001305E5A30D2D11CD97170000938775
:104BC00027A31D8D93070004B397A7004245050452
:104BD0005D8D2AC80C20194617150000130585A104
:104BE000130914002304B102012535C197B7FFFF53
:104BF0009387474195E74247B2471377071009CF9C
:104C000091073EC69257D2973ED225BDB387670320
:104C100085462E84BA9751B79D07E19BA107D5B76A
:104C2000780097060000938666D726860C084E8586
:104C300097000000E7000000FD572A8AE314F5FC06
:104C4000DE2493F70704E39207EC1255C1B5780010
:104C500097060000938686D426860C084E85012A86
:104C6000E1BF797156CA9C49BA8A984522D426D2A6
:104C70004ECE52CC06D64AD05AC85EC6AA892E84D9
:104C8000B284368A63D3E700BA879CC003473404F2
:104C900019C385079CC01C4093F7070281C79C403D
:104CA00089079CC00329040013796900631A09006D
:104CB000130B9401FD5B5C449840998F634CF9049D
:104CC0001C408346340493F70702B336D000A5EBAB
:104CD00013063404D2854E85829AFD576303F5048A
:104CE0001C4011469840998B544481446397C700F7
:104CF000B384E64063D3040081441C4418486354E1
:104D0000F700998FBE94014969047D5B639824057F
:104D1000014509A885465A86D2854E85829A631E2A
:104D200075017D55B250225492540259F249624A9B
:104D3000D24A424BB24B456182800509ADBF330771
:104D4000D40013060003A301C70403475404938748
:104D50001600A2978906A381E7049DBF8546228697
:104D6000D2854E85829AE30E65FB050945B77971B8
:104D700022D426D24AD04ECE06D652CC56CA5AC8D3
:104D8000B689942D930790063289AA842E841386BF
:104D90003504638DF60263E2D706930780056386C8
:104DA000F61863EDD700638E062093073004638EF8
:104DB000F60A930A24042301D404C9A093073006F9
:104DC0006385F60A93074006E395F6FE1C40084308
:104DD00093F6070893054500C5C61C410CC363D86C
:104DE00007001307D002B307F040A301E4049716AD
:104DF00000009386A680294765A893070007638271
:104E0000F61663E5D7029307E0066389F618930761
:104E1000F006E390F6FA0C401C4313F805081385DE
:104E200047006307080608C39C4385A893075007FB
:104E3000E383F6FE930780076389F6129307300732
:104E4000E399F6F61C43D04181459386470014C38D
:104E500083AA07005685492E01C53305554148C030
:104E60005C401CC8A301040461A81C43930A2404E9
:104E7000938647009C4314C32301F4048547D5B7A8
:104E800093F607041C410CC3B9DAC207C18781BF7E
:104E900093F5050408C3C9D99E231307F006638759
:104EA000E60E97060000938666752947A301040461
:104EB0004C400CC463C5050008406D9908C099E3D7
:104EC000B28A89CDB28AB3F5E702FD1AB6958C2174
:104ED0002380BA00B3D5E70263F0E70CA147631E55
:104EE000F7001C40858B91CB58401C4863C7E700F6
:104EF00093070003A38FFAFEFD1A3306564110C82C
:104F00004E87CA867000A2852685EFF09FD57D5A10
:104F1000631D450B7D55B250225492540259F249FB
:104F2000624AD24A424B45618280A382D5049706E9
:104F300000009386A66C0C40084313F805081C413A
:104F40001105630D080208C313F7150001C793E5A7
:104F500005020CC04147B9FB0C4093F5F5FD0CC0B0
:104F6000B1B79C4193E707029CC193078007A30256
:104F7000F404970600009386A66975BF13F805042C
:104F800008C3E30308FCC207C1837DBF9706000086
:104F90009386C666214719BFAE8735B794411C4337
:104FA000CC4913F80608138547006306080008C3B8
:104FB0009C438CC339A008C393F606049C43F5DADE
:104FC0008EA323280400B28A25BF14485686CA85BA
:104FD00026858299E30045F51C40898B8DE7B24711
:104FE0004844E35AF5F23E853DB785465686CA8564
:104FF00026858299E30065F3050A5C443247998F60
:10500000E345FAFEE9BF014A930A94017D5BF5B7D7
:10501000411122C42A842E8597F7FF1F23A00784FD
:1050200006C6EFD09F89FD576319F50097F7FF1F5C
:105030009387C7829C4391C31CC0B2402244410164
:105040008280411122C42E848395E50006C65D2A24
:10505000634905007C48AA977CC8B24022444101BC
:1050600082805E247D777D17F98F5EA4FDB7DE25F3
:10507000011122CC26CA4AC84EC606CE93F70710A5
:10508000AA842E843289B68991C78395E500894622
:1050900001460D225E247D777D17F98F5EA483156E
:1050A000E4006244F240CE864A86B24942492685EF
:1050B000D244056125A8411122C42E848395E500C0
:1050C00006C6CD28FD575A24631AF500FD77FD1753
:1050D000F98F5EA4B2402244410182808567D98F56
:1050E0005EA468C8C5BF8395E50025A8411122C408
:1050F0002A842E85B285368697E7FF1F23A0077680
:1051000006C6EFD0AFF7FD576319F50097E7FF1F0D
:105110009387C7749C4391C31CC0B2402244410191
:105120008280411122C42A842E8597E7FF1F23A77E
:10513000077206C61122FD576319F50097E7FF1F96
:105140009387C7719C4391C31CC0B2402244410164
:105150008280411122C42A842E85B28597E7FF1FE1
:1051600023AE076E06C6CD20FD576319F50097E7FD
:10517000FF1F9387A76E9C4391C31CC0B24022447B
:1051800041018280411122C42A842E8597E7FF1FA6
:1051900023A6076C06C6C920FD576319F50097E7DB
:1051A000FF1F9387A76B9C4391C31CC0B24022444E
:1051B00041018280411122C42A842E85B28536861F
:1051C00097E7FF1F23AC076806C67928FD576319C8
:1051D000F50097E7FF1F938767689C4391C31CC046
:1051E000B24022444101828093F5F50F2A96631460
:1051F000C500014582801C21E38EB7FE0505C5BFB1
:1052000082808280411122C42A842E85B28536860E
:1052100097E7FF1F23A4076406C6B928FD57631943
:10522000F50097E7FF1F938767639C4391C31CC0FA
:10523000B2402244410182809307800517E7FF1F97
:10524000232EF7607D5582809307800517E7FF1FA7
:105250002326F7607D5582809307800517E7FF1F9F
:10526000232EF75E014582809307800517E7FF1F15
:105270002326F75E7D5582809307800517E7FF1F81
:10528000232EF75C7D55828053797374656D436C72
:105290006B3A25640D0A00004368697049443A2559
:1052A0003038780D0A0000005631302E342E36008A
:1052B0004672656552544F53204B65726E656C2083
:1052C00056657273696F6E3A25730D0A000000000F
:1052D00073686F756C646E27742072756E206174CC
:1052E00020686572652121002E2E2F467265655259
:1052F000544F532F706F727461626C652F4D656DE2
:105300004D616E672F686561705F342E6300000029
:10531000657272206174206C696E65202564206F4F
:10532000662066696C6520222573222E200D0A20D6
:10533000000000002E2E2F4672656552544F532FE9
:10534000706F727461626C652F4743432F524953EB
:10535000432D562F706F72742E6300002E2E2F4631
:1053600072656552544F532F71756575652E6300D4
:105370002E2E2F4672656552544F532F7461736BF6
:10538000732E630049444C4500000000F2260000E3
:10539000F2260000322700003E2700008027000090
:1053A000F2260000F2260000322700003E2700000F
:1053B000546D7251000000002E2E2F46726565520A
:1053C000544F532F74696D6572732E630000000093
:1053D000546D72205376630000007A446164632048
:1053E0003A2025642C2025642C2025640A00000026
:1053F000676574534F435077724F6E566F6C74618C
:1054000067653A2025640A00676574496E437572C2
:1054100072656E743A2025640A000000676574495D
:105420006E566F6C746167653A2025640A0000004F
:105430006740533A473C113C6740D33A7461736B01
:1054400031000000BCE8FFFF0EE8FFFF0EE8FFFFA1
:105450000CE8FFFF12E8FFFF12E8FFFFE2E7FFFFA3
:105460000CE8FFFF12E8FFFFE2E7FFFF12E8FFFF93
:105470000CE8FFFFAAE8FFFFAAE8FFFFAAE8FFFF8A
:10548000E2E7FFFF00010202030303030404040434
:1054900004040404050505050505050505050505C0
:1054A00005050505060606060606060606060606A0
:1054B000060606060606060606060606060606068C
:1054C0000606060607070707070707070707070770
:1054D000070707070707070707070707070707075C
:1054E000070707070707070707070707070707074C
:1054F000070707070707070707070707070707073C
:10550000070707070808080808080808080808081F
:10551000080808080808080808080808080808080B
:1055200008080808080808080808080808080808FB
:1055300008080808080808080808080808080808EB
:1055400008080808080808080808080808080808DB
:1055500008080808080808080808080808080808CB
:1055600008080808080808080808080808080808BB
:1055700008080808080808080808080808080808AB
:1055800008080808000000000000000000000000FB
:10559000000000000000000000000000000000000B
:1055A00000000000000000000000000000000000FB
:1055B00000000000000000000000000000000000EB
:1055C00000000000000000000000000000000000DB
:1055D00000000000000000000000000000000000CB
:1055E00000000000232D302B20000000686C4C00D0
:1055F000656667454647000030313233343536370B
:1056000038394142434445460000000030313233CE
:1056100034353637383961626364656600000000EE
:105620000000000000000000010203040607080952
:105630000000000001020304010203040607080938
:1056400000000000060000008025000000000000AF
:10565000000000000000000000000000000000004A
:10566000000000000000000007000000802500008E
:10567000000000000000000000000000000000002A
:105680000000000000000000000000000200000018
:105690008025000000000000000000000000000065
:1056A00000000000000000000000000000000000FA
:1056B000080000008025000000000000000000003D
:1056C00000000000000000000000000000000000DA
:1056D0000000000003000000802500000000000022
:1056E00000000000000000000000000000000000BA
:1056F00000000000000000000500000000C20100E2
:105700000000000000000000000000000000000099
:10571000000000000000000068656C6C6F20776F6F
:10572000726C640A0000000000000000000000002D
:10573000A4550000C455000084550000000000007E
:105740000000000000000000000000000000000059
:105750000000000000000000000000000000000049
:105760000000000000000000000000000000000039
:105770000000000000000000000000000000000029
:105780000000000000000000000000000000000019
:10579000006CDC0202040608AAAAAAAA0E000000F5
:1057A0005C3800200C010020008000200C0100204B
:00000001FF
